:1004B800082910101010101010100821000000005A
:1004C80000000000083F01000100000000000239A0
:0204D800000022
:1005E300E53670207536011203EA8F37E535653736
:1005F300FF5537F534E537F45FF53B853735E5349B
:050603006002F5332246
:10046400E5324531704DF531753201120581E4FBF9
:10047400FA7920784112000E1201F28E398F3A7CFB
:10048400007D641202737C007D0A1202738D29AE12
:1004940039AF3A7C007D0A1202737C007D0A120295
:1004A400738D2A752201AE39AF3A7C007D0A12029F
:0404B400738D2B22F7
:0C06C200754301E4F544F545754601223E
:10069C00538E7F5389F0758A18758CFCC28DD28C61
:0506AC00D2A9D2AF222B
:03000B000203628B
:10036200C0E0C0F0C083C082C0D075D000C000C061
:1003720001C002C003C004C005C006C0070536E5BF
:1003820036B40A037536000532E53270020531FFD4
:10039200AE31BE0109BFF406753100753200053871
:1003A200E538B4080375380074292538F8E6FD7C71
:1003B2000074212538F8E6FB7A00AF381205047480
:1003C2003F2538F8E6FD7C00AF38120546D007D04D
:1003D20006D005D004D003D002D001D000D0D0D0B6
:0803E20082D083D0F0D0E0329C
:1006B10012064B12069C1205E31204641206C28054
:0106C100F543
:10064B00E5A0541F4480F5A07580FF53A01FE5A0C3
:0D065B00541F44A0F5A0E4F58053A01F2219
:0C04DA000108000109FF010AFF010B00EE
:10054600ED4C600FA8077401088002C333D8FC4243
:1005560008800EA8077401088002C333D8FCF45241
:1005660008E50865096013E5A0541F4480F5A0E579
:0A05760008F4F58053A01F85080962
:010580002258
:10060800300005430A108003530AEFE50A650B60C2
:1006180013E5A0541F44A0F5A0E50AF4F58053A003
:040628001F850A0B15
:01062C0022AB
:1004E6001147C0F9A4B0999282F880908883C6A17A
:0D04F600868EFF0858010204081020408087
:10050400E5A0541F44E0F5A07580FF53A01FE5A0AB
:10051400541F44C0F5A074582FF8E6F58053A01F6B
:10052400EB4A600B74472DF8E6547FF5808007741E
:10053400472DF8E6F580E5A0541F44E0F5A053A04C
:020544001F2274
:1003EA00E4FFC2A9C2C4D2C2D2B5D2B420B3027F3A
:1003FA000420B2027F0520B1027F0620B0027F07E7
:10040A00D2C4C2C2D2B5D2B420B3027F0820B2028B
:10041A007F0920B1027F0A20B0027F0BD2C4D2C268
:10042A00C2B5D2B420B3027F0C20B2027F0D20B134
:10043A00027F0E20B0027F0FD2C4D2C2D2B5C2B49C
:10044A0020B3027F1020B2027F1120B1027F122056
:09045A00B0027F13D2A975B0FFB6
:010463002276
:040668007F057E008C
:10066C00EF1FAA0670011E4A600BE4FDEDC3940C4B
:05067C0050EE0D80F7B7
:010681002256
:02062D00A9071B
:10062F00E4FBC294E9139294120668D294E9C313BF
:0C063F00F90BBB08ED7F057E0002066C85
:10068200E4FBC294ECC313FCD29430940343048081
:090692001206680BBB08EBAF0473
:01069B00223C
:1005BC00C201D2947F0C7E0012066CC2947F507ED6
:1005CC000012066CD2947F0A7E0012066CA29492E2
:0605DC0001120668A201F5
:0105E20022F6
:100581001205BC7FCC12062D7F4412062D7FC87E3A
:100591000012066C1205BC7FCC12062D7FBE12061E
:1005A1002D120682A907120682EFAD01FCEC1201A1
:0B05B100B9E4FBFA79807841020117E1
:10000E00EC4D6011E8497017ED33EC3304600DE4EC
:10001E00FCFFFEFD22E933E8330470F802025E12A3
:10002E00022958046009E4CC2481500628500902A4
:10003E000268284003020265C0E0EB4A7044B980B2
:10004E0006D0E0FB020254EF4E701CBD8008EBFFA1
:10005E00EAFEE9FD80EBE98DF0A4FEE5F00200F783
:10006E00E9CDF9EAFEEBFFEF89F0A4FCE5F0CE89CD
:10007E00F0A42EFFE435F0CD89F0A42DFEE435F08A
:10008E008067EF4E7005BD80D780C3EF8BF0A4ACB8
:10009E00F0EE8BF0A42CFCE435F0F8EF8AF0A42CF3
:1000AE00E5F038FCE433CB8DF0A42CFCE5F03BF806
:1000BE00EE8AF0A42CFCE5F038F8E433CF89F0A4F6
:1000CE002CFCE5F038CF3400CE89F0A42FFFE5F0FC
:1000DE003EFEE433C98DF0A42EFEE5F039CD8AF054
:1000EE00A42FFFE5F03EFEE43DFD33D0E0FB5007CC
:1000FE000BBB000F020268EC2CFCEF33FFEE33FE5D
:06010E00ED33FD0202408A
:10011400020268EC5D046005E85904700302025EA3
:10012400120229580460F6EC4860F2EC7004FDFEFB
:10013400FF22C860DB2481C85009C39860025006BE
:100144000202659850CAF582E9294B4A7005AB82D0
:1001540002025475F0007C1A7880C3EF9BEE9AED8E
:1001640099400DC3EF9BFFEE9AFEED99FDE842F036
:10017400DC23ACF0D0E0FFD0E0FED0E0FDAB822089
:10018400E7101BEB60BAEC2CFCEF33FFEE33FEED13
:1001940033FD020240E803F830E705C0F075F000D3
:1001A400EF2FFFEE33FEED33FD40B830E7C280AAF7
:1001B40075F020800E75F010800575F0087D007EC6
:1001C400007F003392D530D5031202C8EC334010BF
:1001D400EF33FFEE33FEED33FDEC33FCD5F0ED22CF
:0E01E400E5F0247EA2D513CC92E7CDCEFF220B
:1001F200EDD2E7CD33EC3392D524814006E4FFFE05
:10020200FDFC22FCE4CFCECDCC24E0501174FF8063
:10021200EDC3CC13CCCD13CDCE13CECF13CF047000
:07022200F030D5DE0202C836
:10022900E9D2E7C933E833F892D5EDD2E7CD33EC1B
:0702390033FC5002B2D52294
:10024000EC30E7100FBF000C0EBE00080DBD00041F
:100250000BEB6014A2D5EB13FCED92E7FD2274FFCB
:10026000FCFDFEFF22E480F8A2D574FF13FC7D8024
:03027000E480EF38
:030000000202D623
:0C02D600787FE4F6D8FD75815F02031DFF
:10027300BC000BBE0029EF8DF084FFADF022E4CC6F
:10028300F875F008EF2FFFEE33FEEC33FCEE9DEC38
:10029300984005FCEE9DFE0FD5F0E9E4CEFD22ED7E
:1002A300F8F5F0EE8420D21CFEADF075F008EF2FC8
:1002B300FFED33FD4007985006D5F0F222C398FDB9
:0502C3000FD5F0EA2256
:0E02C800C3E49FFFE49EFEE49DFDE49CFC2247
:1002E2000206B1E493A3F8E493A34003F68001F27B
:1002F20008DFF48029E493A3F85407240CC8C3331D
:10030200C4540F4420C8834004F456800146F6DFEB
:10031200E4800B01020408102040809004B8E47EBF
:10032200019360BCA3FF543F30E509541FFEE493E0
:10033200A360010ECF54C025E060A840B8E493A3A7
:10034200FAE493A3F8E493A3C8C582C8CAC583CAD2
:10035200F0A3C8C582C8CAC583CADFE9DEE780BE8A
:0105030000F7
:00000001FF
